:1000000089C0AEC05EC3ACC0ABC0AFC0A9C0A8C001
:10001000A7C0A6C0A5C0A4C061C1A2C0A1C081459F
:1000200086468B479048944997609B619E62A16386
:10003000A464A765AA66AC67AE68B069B280B481F3
:10004000B682B883BA84BB84BD84FF21000000005F
:100050000000000000000000000023456C98C9FF6C
:10006000040714233764A0FFFFFFFFFFFFFFFFFF1C
:10007000FFFFFF00000000000000000023405F7A47
:10008000B4FFFFFFFFFFFF001400081400080E1468
:100090000004080E14000305080E140004080A0EDC
:1000A0001114000305080A0E1014000305080A0EB7
:1000B0001012140008000E00080E0004080E0003C1
:1000C00005080E0004080E1100080E1100F3F404D8
:1000D000080E10121400080A0C0E0F10121400085B
:1000E0000EED14000203040500041400040E1400B5
:1000F000040810140004080F1114000305080A0E68
:100100000004080A0E00EEEDECEB140E08040004E7
:10011000080E000011241FBECFE5D2E0DEBFCDBF28
:1001200020E0A0E6B0E001C01D92A437B207E1F7DD
:10013000E5E7F0E085E5808781E083831282118224
:1001400011868BE0828788E58387E1E6F0E08DEF1A
:1001500087838EEF8583712C55245A94C0D0CDC2ED
:100160004FCF1BBC19BC18BC0895189525B7277E26
:1001700025BF29B7226029BF21E022BF019728F0BF
:1001800020E188952150E9F7F9CF089588EE93E0B2
:10019000EDCF369A3699FECF95B1809160008927D0
:1001A000089580917400E3E8F0E080838183828386
:1001B00083830895CF93C72D81E0870D8F73782EA9
:1001C000662D90E08CD26FEF8C2F90E0CF9187C29C
:1001D000FF920F931F93CF93DF93F82E06E710E063
:1001E000CEE7D0E0F11005C0CE0171D2F8018083D6
:1001F00004C0F8016081CE0172D221970F5F1F4FBA
:10020000C337D10579F7DF91CF911F910F91FF90FF
:100210000895D0DF81E0DCCF811101C0A2CF8150F1
:1002200090E0FC01E45BFF4FE491EBBDFC01E05A80
:10023000FF4FE491E9BDFC01EC58FF4F849188BD6C
:1002400008950F931F93CF93C82F8B01CC2359F0A0
:1002500085E0E2DFC8018ADF84DFC80187DFC801EB
:1002600085DFC150F3CFCF911F910F910895EF9289
:10027000FF920F931F93CF93C8E0E82EF12C062F27
:1002800010E084E1C9DFC70171DF6BDFC8016EDFF9
:10029000C150B9F7CF911F910F91FF90EF90089542
:1002A0001F93CF93DF938FEA87B986EC86B91092BC
:1002B000600010E1C0E0D0E085E090E057DF69DF4A
:1002C000C80FD11D1150C1F7CE0124E09695879536
:1002D0002A95E1F7DF91CF911F910895189510921B
:1002E000740087E790E0F3D1853519F0612C91DF38
:1002F00011C0712C872D90E0EAD1682E8F3F19F044
:1003000080E066DF07C0872D21E0270D722E803444
:1003100088F3F6CF80917E008111AB9890917F0099
:100320004091780080917600882311F040E09AE1B6
:100330009F5F80E068E870E0042F10E09923A9F047
:100340009B012F5F3F4FF9013197E491A82FB0E057
:10035000A559BF4FA00FB11FEC93EE2319F0822FC8
:10036000861BEFCF9150B901E9CF840F80938100B4
:10037000442319F091E090936B0080938200962DB6
:10038000953F18F520E12515B0F0209183002F3F0F
:1003900031F407DFE3E8F0E094E09E0F06C09F5FD2
:1003A000692E9817B8F3612CF5CF80818F5F819308
:1003B0009E13FBCF0AC0F5DE80917600811104C048
:1003C00080917700811101C0612C512C8FEF8DBD80
:1003D00080E68CBDAB9A8FE384BB8BE187BB8CEE50
:1003E00088BB81E083BF91EA9ABD80BF8BB78062F2
:1003F0008BBF8AB785608ABF85B7806285BF7894D6
:100400008CE287B986EC86B93699FECF8FEF809360
:100410006000C62DC53F10F0612C39C0809183006B
:10042000803138F4E62DF0E0E559FF4FC081DC2F34
:100430002EC0ACDEB6DEC6E7D0E000E010E0FF2460
:10044000F39481E0800F0F5F1F4F98819F3F29F445
:10045000219609301105A9F7E5CF6DE570E0F1DED1
:10046000F801EF59FF4F608088818F258883D1DEA6
:100470006FE070E080E2E5DE88818F258883612C63
:10048000C8DE84DE80917600882311F3CBCF92DE24
:1004900010E0F12C8CE2D82E96ECC92EEE24EA94D2
:1004A000CE3E19F463E481E204C0CD3E21F468E25B
:1004B00084E1DDDE76C0CC3E11F469E203C0CB3EC0
:1004C00019F462E581E0F5CFC33F81F404E084E1F3
:1004D000A3DE85E090E04ADE88E09EDE81E490E0E5
:1004E00045DE0150A1F780ED92E05AC0C43F51F5BE
:1004F00084E690E03BDE4DDE90E0292F30E0F9010C
:10050000E25EFF4FE491E81710F49E5FF6CFF90129
:10051000E15EFF4F04916DE770E0802F8295869534
:1005200087708FDE8EEE92E021DE65E070E081E084
:1005300088DE85E694E01ADE6DE770E0802F8F712B
:1005400080DE0DC0CE3F71F400E000937F0061DEDD
:100550006AEF70E081E075DE0F5F0A31B1F716DEF9
:1005600015DE1FC0CD3F51F58FEF8093800051DE27
:1005700085E052DE0BDE0ADE84E14EDE91DE809302
:10058000800047DE03DE02DEF9CF3699FECFE0922F
:100590006000F394909180008917B0F484EF91E0AB
:1005A000E5DDFFDDF6DD803998F51F5F183008F4D2
:1005B00077CFD53190F010E0DAE0CAE08D2F2CDE55
:1005C0006FDED7B8C6B8E1CFDB3040F384E18F15DA
:1005D00028F7E0927400DAE0E1CFD23030F08D2FCE
:1005E00086958695D695D80F12C0BBDD85B7877ED8
:1005F000806185BFF89485B7846885BF8B7F85BF90
:1006000085B7806285BF889585B78F7D85BFCD2FE3
:1006100010E046CF112416B8A4DD87B38C7E87BBCB
:1006200080E051E041E020E030E0A8E0999B06C086
:10063000F9013197F1F79AB795609ABF96B39A2767
:10064000999B03C0511003C034C0911107C040E30F
:10065000451588F581112FC050E049E0652D71E006
:10066000623308F070E0760F572E511108C08111E7
:1006700005C081E0911103C080E001C081E099983C
:1006800095B7977E906195BFA895942F987011F4B7
:1006900090E401C090E6916091BD95B7946895BFD4
:1006A0009B7F95BF78948895F89491B59F7B91BD79
:1006B000BDCF9111D3CF8FE58DBF82E08EBF1FBE1E
:1006C0000EDE999A552011F0189501C0A3DFE1992B
:1006D000FECF9FBB8EBBE09A99278DB30895262F3E
:1006E000E199FECF1CBA9FBB8EBB2DBB0FB6F89411
:0E06F000E29AE19A0FBE01960895F894FFCFAA
:00000001FF
